:100000000C9434000C9451000C9451000C94510049
:100010000C9451000C9451000C9451000C9451001C
:100020000C9451000C9451000C9451000C9451000C
:100030000C9451000C9451000C9451000C945100FC
:100040000C9451000C9451000C9453000C945100EA
:100050000C9451000C9451000C9451000C945100DC
:100060000C9451000C94510011241FBECFEFD8E026
:10007000DEBFCDBF13E0A0E0B1E0E8E7F5E002C0ED
:1000800005900D92A030B107D9F714E0A0E0B3E0DD
:1000900001C01D92A431B107E1F70E9451010C94F7
:1000A000BA020C9400001F920F920FB60F92112407
:1000B0008F939F93EF93FF9380911304813049F5C1
:1000C00080910003E82FF0E09091C600E857FC4FC4
:1000D00090838F5F8093000380910003843091F5BB
:1000E0001092000380918803809387038091890395
:1000F00080930E0480918A038093060380918B0382
:1001000080938C03809187038C34E1F41092130464
:1001100019C0809113048823A9F480910003E82F6B
:10012000F0E09091C600E357FC4F90838F5F80937F
:10013000000380910003803829F41092000381E0CD
:1001400080931304FF91EF919F918F910F900FBEB9
:100150000F901F90189530918C0320910603809189
:100160000E0490E0A0E0B0E0DC0199278827830F1F
:10017000911DA11DB11D522F40E060E070E0840F81
:10018000951FA61FB71F80930F0490931004A09390
:100190001104B0931204089580910F0490911004FB
:1001A000A0911104B09112044091020350910303F5
:1001B0006091040370910503840F951FA61FB71F5C
:1001C0008093020390930303A0930403B093050369
:1001D000EA2FE695E0930D04F0E0E95FFC4F8081A3
:1001E00085B9809187038234B9F6089589E18093B7
:1001F000C4001092C50088E98093C10010920003EA
:1002000008959091C00095FFFCCF8093C60008959B
:100210008091C00087FFFCCF8091C6000895829531
:1002200090E09C0123733070220F331F220F331F85
:100230008C7C90709595879595958795282B30E0C7
:10024000C90185759070880F991F2A7A307035958D
:100250002795822B0895EF92FF920F931F93CF93D0
:10026000DF930F92CDB7DEB78C0190E0E92EFF242B
:10027000F801EE0DFF1D8081880F880F99830E9481
:100280000F01F701E95FFC4F808399819F5F9038F0
:1002900069F70F90DF91CF911F910F91FF90EF9031
:1002A00008958FEF84B90E94F600789482E48093D9
:1002B000870381E080931304CAE287EA91E60197FD
:1002C000F1F700C00000809187038335A1F51092FB
:1002D00002031092030310920403109205030E947C
:1002E000AB0084E40E94010184E40E94010183E5E3
:1002F0000E9401018FE50E94010183E50E94010136
:1003000089E60E9401018EE60E9401018FE50E94AC
:10031000010183E50E94010185E60E94010184E755
:100320000E9401018DE00E9401018AE00E9401010A
:1003300080E892E0F1C0809187038435A1F51092A6
:1003400002031092030310920403109205030E940B
:10035000AB0084E40E94010184E40E94010183E572
:100360000E9401018FE50E94010184E50E940101C4
:1003700082E70E94010189E60E9401018FE50E9447
:10038000010183E50E94010185E60E94010184E7E5
:100390000E9401018DE00E9401018AE00E9401019A
:1003A00080E092E0B9C0809187038535E9F510922D
:1003B00002031092030310920403109205030E949B
:1003C000AB0084E40E94010184E40E94010183E502
:1003D0000E9401018FE50E94010182E50E94010156
:1003E00081E60E9401018DE60E94010180E70E94E2
:1003F000010185E50E94010180E70E9401018FE56E
:100400000E94010183E50E94010185E60E9401012D
:1004100084E70E9401018DE00E9401018AE00E94B0
:10042000010180E891E078C0809187038434E9F588
:10043000109202031092030310920403109205031A
:100440000E94AB0084E40E94010184E40E94010147
:1004500083E50E9401018FE50E94010182E50E946F
:10046000010181E60E9401018DE60E94010180E701
:100470000E94010184E40E9401018EE60E940101B4
:100480008FE50E94010183E50E94010185E60E943B
:10049000010184E70E9401018DE00E9401018AE0D0
:1004A0000E94010180E091E037C080918703813490
:1004B000C1F51092020310920303109204031092EC
:1004C00005030E94AB0084E40E94010184E40E94C1
:1004D000010183E50E9401018FE50E94010181E491
:1004E0000E94010182E70E94010182E60E9401014F
:1004F0008FE50E94010183E50E94010185E60E94CB
:10050000010184E70E9401018DE00E9401018AE05F
:100510000E9401018DE893E00E942B010E94CC0013
:10052000CCCE80918703893409F0C7CE81E40E9444
:1005300001018AE60E9401018FE50E94010183E525
:100540000E94010189E60E94010187E60E940101E3
:1005500087E40E94010185E60E9401018EE60E9467
:1005600001018DE00E9401018AE00E940101C09317
:080570008703A3CEF894FFCF2E
:100578003F3E3E3D3D3C3C3B3B3A3A3939383837C3
:100588003736363535343433333232313130302F33
:100598002F2E2E2D2D2C2C2B2B2A2A2929282827A3
:1005A8002726262525242423232222212120201F13
:1005B8001F1E1E1D1D1C1C1B1B1A1A191918181783
:1005C8001716161515141413131212111110100FF3
:1005D8000F0E0E0D0D0C0C0B0B0A0A090908080763
:1005E80007060605050404030302020101000000D2
:1005F80000000001010202030304040505060607C2
:1006080007080809090A0A0B0B0C0C0D0D0E0E0F32
:100618000F101011111212131314141515161617A2
:1006280017181819191A1A1B1B1C1C1D1D1E1E1F12
:100638001F20202121222223232424252526262782
:1006480027282829292A2A2B2B2C2C2D2D2E2E2FF2
:100658002F30303131323233333434353536363762
:1006680037383839393A3A3B3B3C3C3D3D3E3E3FD2
:100678001F202122232425262728292A2B2C2D2E0A
:100688002F303132333435363738393A3B3C3D3EFA
:100698003F3E3D3C3B3A39383736353433323130DA
:1006A8002F2E2D2C2B2A29282726252423222120CA
:1006B8001F1E1D1C1B1A19181716151413121110BA
:1006C8000F0E0D0C0B0A09080706050403020100AA
:1006D80000000102030405060708090A0B0C0D0EA9
:1006E8000F101112131415161718191A1B1C1D1E9A
:1006F8001F2122242527282A2B2D2E30313233354D
:10070800363738393A3A3B3C3D3D3E3E3E3F3F3F27
:100718003F3F3F3F3E3E3E3D3D3C3B3A3A3938370E
:100728003635333231302E2D2B2A28272524222105
:100738001F1E1C1B191816151312100F0E0C0B0A6E
:100748000908070605040303020101000000000070
:100758000000000000000101020303040506070869
:10076800090A0B0C0E0F101213151618191B1C1E54
:00000001FF
